:1000000090C0B4C0B3C0B2C0B1C019C7AFC0AEC019
:10001000ADC0ACC0ABC0AAC0A9C0A8C0A7C097A0C3
:10002000895B5A0F830DC95F6035C2E907E18C24F3
:10003000671E458E086325F0150A17BE0694F778EB
:10004000EA4B001AC53E5EFCDBCB75230B2039B1B1
:100050002158ED953857AE147D88ABA844AF4AA51A
:1000600047868B301BA64D929EE7536FE57A3CD3B3
:1000700085E6DC695C29372EF528F4668F36411950
:100080003FA101D85049D14C84BBD05912A9C8C452
:10009000878274BC9F56A4646DC6ADBA034034D940
:1000A000E2FA7C7B05CA2693767EFF5255D4CFCEEA
:1000B0003BE32F103A11B6BD1C2ADFB7AAD577F85B
:1000C00098022C9AA346DD99659BA72BAC09811653
:1000D00027FD13626C6E4F71E0E8B2B97068DAF612
:1000E00061E4FB22F2C1EED2900CBFB3A2F1513316
:1000F00091EBF90EEF6B31C0D61FB5C76A9DB854AE
:10010000CCB07379322D7F0496FE8AECCD5DDE7221
:10011000431D1848F38D80C34E42D73D9CB49700D1
:10012000690711241FBECFE5D2E0DEBFCDBF10E0CE
:10013000A0E6B0E0EEEAF5E102C005900D92A03B2A
:10014000B107D9F721E0A0EBB0E001C01D92A431C6
:10015000B207E1F710E0C1E9D0E003C02197FE014A
:100160001ADAC039D107D1F7C4D61FCA49CF80E9FE
:1001700091E008953FB7F8948091B7009091B8004E
:10018000A091B900B091BA0022B708B601FE05C02F
:100190002F3F19F00196A11DB11D3FBFBA2FA92F06
:1001A000982F8827BC01CD01620F711D811D911D03
:1001B00042E0660F771F881F991F4A95D1F708956F
:1001C000CF92DF92EF92FF92CF93DF936B017C018E
:1001D000D1DFEB01CFDF6C1B7D0B683E7340A0F0DD
:1001E000C114D104E104F10439F4DF91CF91FF90FF
:1001F000EF90DF90CF90089581E0C81AD108E10810
:10020000F108C851DC4FE6CFC114D104E104F10478
:1002100009F7EBCF2FB7F8946091B3007091B40059
:100220008091B5009091B6002FBF08952F923F9214
:100230004F925F927F928F929F92AF92BF92CF9296
:10024000DF92EF92FF920F931F93CF93DF9300D033
:100250001F92CDB7DEB7E090070180910A0190911F
:100260000B01A0910C01B0910D01892B8A2B8B2BD6
:10027000D1F080DF0091030110910401209105016C
:1002800030910601601B710B820B930B00910A01E8
:1002900010910B0120910C0130910D016017710735
:1002A00082079307D0F266DF609303017093040125
:1002B0008093050190930601E0911201F0911301E2
:1002C000309759F040910E0150910F01609110014B
:1002D000709111018E2D0995E82E00910101109168
:1002E00002012E2C312C512C412C0115110509F441
:1002F0005CC0D8011C967C901C978091080190915D
:1003000009018436910510F41C961C92D801ED91D8
:10031000FC918280938019821A821B82EE2079F1EF
:100320005801B6E0AB0EB11CD12CC12CF501619186
:100330005F016623E9F0F280FF20D1F070E090E0E9
:1003400080E06F5F7F4F8F4F9F4FA201910194D844
:100350002F2D30E050E040E02F5F3F4F4F4F5F4F79
:100360008BD8E1E0F0E0EC0FFD1FEC0DFD1D80836C
:10037000FFEFCF1ADF0A23E0C216D104B9F6D80185
:100380001D964D915C911E9712966D917C919E01E8
:100390002F5F3F4FC801F4010995D8011C967C924C
:1003A0001C9714960D911C91A0CF8091FF00909105
:1003B00000017C01BFEFEB1AFB0AF0920001E09212
:1003C000FF004997B4F126DF0091FB001091FC007B
:1003D0002091FD003091FE005B016C01A01AB10A72
:1003E000C20AD30A960185010115110521053105BF
:1003F00021F401E010E020E030E0C70168EE73E096
:1004000092D8BC01990F880B990BA901980169D862
:100410003093090120930801109200011092FF000F
:10042000F9DE6093FB007093FC008093FD009093D5
:10043000FE000F900F900F90DF91CF911F910F91C1
:10044000FF90EF90DF90CF90BF90AF909F908F90F4
:100450007F905F904F903F902F900895282F87FDB9
:100460008095682F70E0CB0101965DD8892F880FA9
:1004700027FD80950895BF92CF92DF92EF92FF9271
:100480000F931F93CF93DF93D62E092F10E0F8011F
:10049000E25EFF4F2491270F30E0F901E25EFF4F4B
:1004A000E490F901E15EFF4FD491015E1F4FF80126
:1004B0000491700F072F10E0F801E25EFF4FC49126
:1004C000015E1F4FF8010491182F1695F62EF69431
:1004D000CF2CC4DFB82E8D2DC1DFD82E40E8410FC0
:1004E000EC2FF0E0E25EFF4F9491242F3F2D92FD20
:1004F00002C02F2D342F90FD319591FD219525952A
:100500003595321FEE2DF0E0E25EFF4FE491212F92
:10051000E2FF02C02F2DC12EE0FD2195E1FDC19427
:100520005C2D55952595251FAB2DB0E01196231711
:100530000CF04DC0321B832F90E0BD01F4D7290F82
:1005400030E83F0DE02FF0E0E25EFF4FE491532FE3
:10055000E2FF02C0542F432FE0FD4195E1FD51958C
:1005600055954595451FED2FF0E0E25EFF4FE49174
:10057000E2FF03C0812F132F382FE0FD1195E1FD1D
:10058000319535951595131F141744F5411B842F8C
:1005900090E0BD01C8D7910F6D2D70E06F5F7F4F68
:1005A000291724F5921B892F90E0BDD7920F905CFC
:1005B000292F220F08F42FEF822FDF91CF911F9167
:1005C0000F91FF90EF90DF90CF90BF900895822F12
:1005D000831B90E0BD01A7D7291BB2CF812F841BBD
:1005E00090E0BD01A0D7191B912FD6CF822F891B78
:1005F00090E099D7291B922FDACFCF93DF93EC01AC
:10060000DB014881E981FA81C42FCC0FCC0FCC0FDC
:10061000D0E0CE0166E570E086D7292F842F807464
:10062000342F307247FD78C0811165C0311105C08B
:10063000892F8095492F282F04C045E5490F30E0C8
:100640002BEAEF3F39F1EE2309F484C0222339F07D
:100650008E2F90E0622F70E0019665D7292F4423FA
:1006600039F08E2F90E0642F70E001965CD7492F0F
:10067000332339F08E2F90E0632F70E0019653D72B
:10068000392FE0956E2F70E0CB0101964CD7290FE2
:10069000490F390FFF3F31F16F2F70E0CB0143D786
:1006A000E1E0F11101C0E0E0E90F09F457C02223B5
:1006B00039F08E2F90E0622F70E0019634D7292F09
:1006C000442339F08E2F90E0642F70E001962BD7F1
:1006D000492F332339F08E2F90E0632F70E001967D
:1006E00022D7392F2C9311964C93119712963C9345
:1006F000DF91CF910895311109C0CE016BEA70E00E
:1007000012D78BEA891B4AEA420F95CF80E0492F26
:100710004095392F20E095CF81110FC0311109C0CC
:10072000CE016BEA70E0FFD64BEA491B35E5390F85
:10073000F1CF392F309540E084CF311106C085E5E7
:10074000890F3BEA321B282FF6CF8AEA890F90E007
:1007500035E5F8CF3FEF4FEF2FEF9CCF30E040E093
:1007600020E0C0CFEF92FF920F931F93CF93DF93C0
:100770003091B1003F5F232F27702093B100C0E874
:1007800030FFC0E021FDC064247009F0C062C05F8A
:10079000FC018C010D5F1F4FE12CFF24F394D0E08E
:1007A0002485222331F0622F70E0C701CDD621E0ED
:1007B000260F2187822F90E00196BE01B4D69111B9
:1007C00011C01682222319F06FEF620F61873196F4
:1007D0000E171F0729F7DF91CF911F910F91FF90FF
:1007E000EF90089591509683EDCF4F925F926F9264
:1007F0007F928F92AF92BF92CF92DF92EF92FF9251
:100800000F931F93CF93DF933C01EB01B3DCF30114
:1008100027853089621B730B6A307105B8F3F89431
:10082000E881F98158B3546048B34B7F48BBC98411
:100830008E812C2D281B822F2E83BF844A805B80C3
:100840006C857D85DE846F5F7F5FD3949F81388563
:10085000AA84EB841081D20120E0C32F022F322F13
:100860003081112788943111380F08F43FEF8195BA
:10087000889460FD130F1795889461FD130F1795E9
:10088000889462FD130F1795889463FD130F1795D5
:10089000889464FD130F1795889465FD130F1795C1
:1008A000889466FD130F1795889467FD130F1795AD
:1008B0008894232F6111212F8C0D122F002C58BBEF
:1008C00000C017FF48BB31812227889400C000C0B8
:1008D000002C48BB3111390F00C0002C58BB00C0A0
:1008E00016FF48BB08F43FEF9195889400C000C004
:1008F000002C48BB70FD230F00C0002C58BB00C06B
:1009000015FF48BB2795889471FD230F00C000C0D8
:10091000002C48BB2795889400C0002C58BB00C011
:1009200014FF48BB72FD230F2795889400C000C0B8
:10093000002C48BB73FD230F00C0002C58BB00C027
:1009400013FF48BB2795889474FD230F00C000C097
:10095000002C48BB2795889400C0002C58BB00C0D1
:1009600012FF48BB75FD230F2795889400C000C077
:10097000002C48BB76FD230F00C0002C58BB00C0E4
:1009800011FF48BB2795889477FD230F00C000C056
:10099000002C48BB2795889400C0002C58BB00C091
:1009A00010FF48BB132F7111122F9A0D00C000C009
:1009B000002C48BB00C000C0002C58BB00C017FF73
:1009C00048BB32812227889400C000C0002C48BB5D
:1009D00031113C0F00C0002C58BB00C016FF48BBB3
:1009E00008F43FEFEB0DF11D00C000C0002C48BB28
:1009F000D0FC230F00C0002C58BB00C015FF48BB23
:100A000027958894D1FC230F00C000C0002C48BB60
:100A10002795889400C0002C58BB00C014FF48BB29
:100A2000D2FC230F2795889400C000C0002C48BB3F
:100A3000D3FC230F00C0002C58BB00C013FF48BBE1
:100A400027958894D4FC230F00C000C0002C48BB1D
:100A50002795889400C0002C58BB00C012FF48BBEB
:100A6000D5FC230F2795889400C000C0002C48BBFC
:100A7000D6FC230F00C0002C58BB00C011FF48BBA0
:100A800027958894D7FC230F00C000C0002C48BBDA
:100A90002795889400C0002C58BB00C010FF48BBAD
:100AA000132FD110122FC19500C000C0002C48BBDD
:100AB000CE0D00C000C058BB00C017FF48BB30813E
:100AC0002227889400C000C0002C48BB3111380F89
:100AD00000C0002C58BB00C016FF48BB08F43FEF15
:100AE0008195889400C000C0002C48BB60FD230F96
:100AF00000C0002C58BB00C015FF48BB2795889448
:100B000061FD230F00C000C0002C48BB27958894CE
:100B100000C0002C58BB00C014FF48BB62FD230F6F
:100B20002795889400C000C0002C48BB63FD230FAC
:100B300000C0002C58BB00C013FF48BB2795889409
:100B400064FD230F00C000C0002C48BB279588948B
:100B500000C0002C58BB00C012FF48BB65FD230F2E
:100B60002795889400C000C0002C48BB66FD230F69
:100B700000C0002C58BB00C011FF48BB27958894CB
:100B800067FD230F00C000C0002C48BB2795889448
:100B900000C0002C58BB00C010FF48BB132F6111D0
:100BA000122F8C0D00C000C0002C48BB119709F01B
:100BB00086CEB201052C000C880B990B20EE31E09B
:100BC00040E050E059D46B017C01F4E0F694E794E6
:100BD000D794C794FA95D1F7C2016BE970E0A3D41A
:100BE000292F30E0D701C601820F931FA11DB11D2F
:100BF000893EE3E09E07A105B10590F1885E934030
:100C0000A109B10922E0B695A795979587952A95F0
:100C1000D1F79C0143E0220F331F4A95E1F7232FC0
:100C200033276091B00070E0860F971F820F931FEB
:100C30004091B3005091B4006091B5007091B6003E
:100C4000292F3327420F531F611D711D4093B3009D
:100C50005093B4006093B5007093B6008093B000D9
:100C6000789488DAF301708B6787DF91CF911F91B9
:100C70000F91FF90EF90DF90CF90BF90AF908F904B
:100C80007F906F905F904F900895BA9A08950F9358
:100C90001F93CF93DF93CDB7DEB762970FB6F8946B
:100CA000DEBF0FBECDBF8C01F901DC011C968C911B
:100CB0007A8369835C834B835E834D8390819D87B8
:100CC00091819E8792819F878130E9F4CE010196C0
:100CD00049DD83E0888B1A8A198AD801ED91FC914D
:100CE0000484F585E02DBE016F5F7F4FC801099533
:100CF00062960FB6F894DEBF0FBECDBFDF91CF91E5
:100D00001F910F9108951C861B861A8619861886D6
:100D10001F82DFCF0F931F93CF93DF93CDB7DEB743
:100D200062970FB6F894DEBF0FBECDBF8C01F901FC
:100D3000DC011C968C917A8369835C834B835E8390
:100D40004D8390819D8791819E8792819F8781307D
:100D5000E1F4CE01019606DD188A1A8A198AD801B3
:100D6000ED91FC910484F585E02DBE016F5F7F4F0E
:100D7000C801099562960FB6F894DEBF0FBECDBFCD
:100D8000DF91CF911F910F9108951C861B861A86C3
:100D9000198618861F82E0CF90E080E00895FC015C
:100DA000858596850895CF93DF9300D000D000D03D
:100DB000CDB7DEB7AB011C821D821E82DC01ED9136
:100DC000FC910190F081E02D19821A821B829E0114
:100DD0002F5F3F4FBE016C5F7F4F099526960FB680
:100DE000F894DEBF0FBECDBFDF91CF910895809103
:100DF000E4009091E500A091E600B091E700B4997D
:100E00000CC00196A11DB11D8093E4009093E500F4
:100E1000A093E600B093E700EACF1092E4001092AE
:100E2000E5001092E6001092E700813A9648A14052
:100E3000B10514F081E0089580E00895B2D31F92C7
:100E40000F920FB60F9211242F933F938F939F937E
:100E5000AF93BF938091B3009091B400A091B5007F
:100E6000B091B6003091B20023E0230F2D3768F126
:100E700026E8230F0296A11DB11D2093B200809396
:100E8000B3009093B400A093B500B093B6008091E6
:100E9000B7009091B800A091B900B091BA00019646
:100EA000A11DB11D8093B7009093B800A093B90025
:100EB000B093BA00BF91AF919F918F913F912F91C5
:100EC0000F900FBE0F901F9018950196A11DB11D98
:100ED000D4CFE7E0F1E08FEF808312821182148695
:100EE00013868FEF9FEFDC0187839087A187B287FE
:100EF00091C9CF93DF9300D01F92CDB7DEB783E0C7
:100F00008ABD83BF789489B7826089BF80E48CBD35
:100F10008FEF8DBD97EC90BF97E896B99091CE007A
:100F2000911144C01092C0001092BF008093C30082
:100F30008093C4008093C5008093C6008093C7004F
:100F40008093C80081E08093C9001092CB0010927A
:100F5000CA001092C2001092C100809101019091CC
:100F60000201892B31F48DEB90E090930201809384
:100F70000101E091BB00F091BC00309721F08DEBB6
:100F800090E0958384838DEB90E09093BC008093F8
:100F9000BB001092CD001092CC0081EA90E09093BB
:100FA000BE008093BD0081E08093CE00BA9A88EEA7
:100FB00090E09093C0008093BF0086E090E0909313
:100FC000CB008093CA0080910A0190910B01A091FF
:100FD0000C01B0910D01843C29E09207A105B105F7
:100FE00020F484EC99E0A0E0B0E080930A019093B3
:100FF0000B01A0930C01B0930D018FB7F894BC982E
:10100000C4988FBFDD24DA949AE0C92E412C512C6C
:1010100032014A943AEF232E30E0332E8091FA00C9
:10102000823009F4A0C0F8F4882309F444C0813068
:1010300009F451C0DCDE882381F08091FA008F5FD3
:10104000853008F074C18093FA001092E400109289
:10105000E5001092E6001092E7006EE170E080E09B
:1010600090E0AED8DBCF833009F4D2C0843011F7E2
:10107000C0920701FF24F39408EE10E0F982DA82AF
:10108000DB82B801CE010196B8DA0D5F1F4F20E078
:101090000A3F120799F7CAD8AADE882309F43EC18D
:1010A00064EF71E080E090E08BD8A1DE8823E9F363
:1010B0001092FA00BFCF08EE10E019821A821B824C
:1010C000B801CE01019699DA0D5F1F4F2016310647
:1010D000A1F7ACD8AFCF9ED80091DA001091DB0019
:1010E0002091DC003091DD00601B710B820B930BB3
:1010F000643671058105910508F49CCF8BD8609307
:10110000DA007093DB008093DC009093DD00109296
:10111000D6001091D6001630B0F4812F90E0FC017B
:10112000E05AFF4F20812983DA82DB8263E070E09E
:10113000FAD1BC0168517F4FCE0101965EDA1F5F84
:101140001093D600E6CFC092070170D88091870037
:10115000E7E8F0E09291918390E0E036F907D1F76B
:101160008093600067CF56D80091DA001091DB00C1
:101170002091DC003091DD00601B710B820B930B22
:101180006A3071058105910508F454CF43D8609306
:10119000DA007093DB008093DC009093DD00909187
:1011A000D900809188002091D8009217B9F09983D6
:1011B000DA822AEF2B8390E063E070E0B4D1BC01C7
:1011C00068517F4FCE01019618DAC09207012ED8E0
:1011D0008091D9008F5F8093D9002CCF2091D700C8
:1011E0002093D900882321F081508093880022CF5A
:1011F00085E0809388009093D7009093D900E5D044
:101200002AEF30E040E050E050D16093D80012CF98
:101210009EE190930701FED70091E0001091E1005C
:101220002091E2003091E300601B710B820B930B65
:10123000653171058105910508F4FCCEEBD760930B
:10124000E0007093E1008093E2009093E30088EE69
:10125000A82E80E0B82EF12CE12C0091DE00109138
:10126000DF00B801C70107D9B801C70104D9B80127
:10127000C70101D9982EB801C701FDD8B801C7012F
:10128000FAD8B801C701F7D8882EB801C701F3D83A
:10129000682F70E090E080E025E130E040E050E031
:1012A000EBD0A301920101D1205B2983682D70E06E
:1012B00090E080E026EF3FEF4FEF5FEFDDD0A3013E
:1012C0009201F3D021503F4F4F4F5F4F2A83692D3A
:1012D00070E090E080E029EB30E040E050E0CCD0DE
:1012E000A3019201E2D02A5B3F4F4F4F5F4F2B8308
:1012F000B501CE01019681D92FE0E20EF11C83E009
:10130000A80EB11C9AE5E916F10409F0A6CF0C5E0F
:101310001F4F1093DF000093DE00DBCE62E370E02E
:1013200080E090E04DD7F394F110A6CE83CE1092DA
:10133000FA008BCE8F929F92AF92BF92CF92DF92A4
:10134000EF92FF92CF93DF93EC01688179818A81DC
:101350009B81611571058105910521F464E279EDA8
:101360008BE597E02DE133EF41E050E09ED049015D
:101370005A0127EA31E440E050E07ED06B017C0165
:101380002CEE34EF4FEF5FEFC501B40175D0C60E00
:10139000D71EE81EF91EF7FE06C081E0C81AD10864
:1013A000E10880E8F80AC882D982EA82FB82C70194
:1013B000B6019F77DF91CF91FF90EF90DF90CF90B4
:1013C000BF90AF909F908F9008958F929F92AF9211
:1013D000BF92CF92DF92EF92FF926091890070915D
:1013E0008A0080918B0090918C00611571058105B8
:1013F000910521F464E279ED8BE597E02DE133EF7F
:1014000041E050E052D049015A0127EA31E440E07E
:1014100050E032D06B017C012CEE34EF4FEF5FEFE8
:10142000C501B40129D0C60ED71EE81EF91EF7FE6D
:1014300006C081E0C81AD108E10880E8F80AC09225
:101440008900D0928A00E0928B00F0928C00C70154
:10145000B6019F77FF90EF90DF90CF90BF90AF9055
:101460009F908F9008956093890070938A00809375
:101470008B0090938C000895EE27FF27AA27BB27A7
:1014800008C0A20FB31FE41FF51F220F331F441F14
:10149000551F969587957795679598F37040A9F7AE
:1014A000009799F7BD01CF010895052E97FB16F41B
:1014B00000940FD057FD05D014D007FC02D046F49D
:1014C00008C050954095309521953F4F4F4F5F4F45
:1014D000089590958095709561957F4F8F4F9F4FA0
:1014E0000895A1E21A2EAA1BBB1BFD010DC0AA1F65
:1014F000BB1FEE1FFF1FA217B307E407F50720F07D
:10150000A21BB30BE40BF50B661F771F881F991FF7
:101510001A9469F760957095809590959B01AC0140
:10152000BD01CF0108950024552704C0080E591F9E
:10153000880F991F009729F076956795B8F3710584
:10154000B9F7802D952F089597FB072E16F4009478
:1015500006D077FD08D00BD007FC05D03EF490955F
:1015600081959F4F0895709561957F4F0895AA1BAF
:10157000BB1B51E107C0AA1FBB1FA617B70710F07E
:10158000A61BB70B881F991F5A95A9F780959095B0
:10159000BC01CD010895EE0FFF1F0590F491E02DE1
:0E15A000099481E090E0F89400C0F894FFCF29
:1015AE0000060C12181E242A30363C42484E545A5D
:1015BE0060666C72787E848A90969CA2A8AEB4BA4D
:1015CE00C0C6CCD2D8DEE4EA05010000000000005F
:1015DE00001E071E071E07D306CF06CC060000000E
:1015EE00008A0647064506D306CF06B700F5030068
:00000001FF
